:020000020000FC
:0200000054C0EA
:0200140049C3DE
:02001800F5C130
:02003C0078C288
:020074006EC25A
:0200900000C4AA
:1000A80039C201E20EBF0FEF0DBF07E104B908E046
:1000B80005B901E00DBD00E50CBD289A2C98179AEA
:1000C8000F9A0CE000936A0000E20DBBEE27CC27E4
:1000D800F2E0D2E0B5E0AA277FEF84E054E039D11E
:1000E80003EC289843D104E041D1289A000000008D
:1000F80000000000000000000000000000000000F8
:10010800000000000000000000005FEF22D101E0C5
:1001180000937E0000EC00937C0006E005BD00E241
:100128000093B60007E00093B1000091B6000F718C
:10013800E1F7002707BB01E00093700000E000939F
:10014800A90000E10093A800689A749807D208E90A
:100158000093C9000CE00093CC005DD000EE289815
:1001680005D10FEF03D1289A01EE2898FFD00AEAAB
:10017800FDD0289A02EE2898F9D00DECF7D0289AED
:1001880003EE2898F3D00BEAF1D0289A08EC2898C7
:10019800EDD006E3EBD0289A05EC2898E7D000E8E4
:1001A800E5D0289A0CEE2898E1D008E3DFD0289A09
:1001B8000EEE2898DBD007E0D9D0289A0DEE2898C3
:1001C800D5D008EFD3D0289A0EEC2898CFD008E0E5
:1001D800CDD0289A0FE82898C9D0289A00270CBBB8
:1001E800789437D0FD1303C0EC1301C0FBCF2FEF79
:1001F8008AD12191122E87D1219185D11A94E1F7C4
:100208002FEF81D12AEA7FD12EEF7DD12DEF7BD13F
:10021800F2FDF2E0E7CF02EC2898A8D008E0A6D0DB
:10022800289A01E82898A2D000E0A0D0289A08309F
:10023800C1F7089502EC289899D009E097D0289A38
:1002480001E8289893D000E091D0289A0930C1F7A6
:10025800089502EC28988AD006E188D0289A01E807
:10026800289884D000E082D0289A0631C1F70895F2
:1002780002EC28987BD009E179D0289A01E82898DF
:1002880075D000E073D0289A0931C1F7089507E8BE
:1002980028986CD000E06AD0902E289A00E228981E
:1002A80065D000E063D0065009930350002E00E0AB
:1002B8005DD000E05BD000E059D009930A9501F4C5
:1002C80000E054D000E052D000E050D000E04ED022
:1002D80000E04CD009930A94D9F700E047D000E039
:1002E80045D000E043D0289A09939992D2FDD2E0F4
:1002F8000895B5DF9FDF0FE8289838D000E036D0A2
:10030800289A03FDC4DFB4DF2C9A00002C9800E67D
:1003180028982CD00D91902F18E0010F27D001E6D6
:1003280025D008E823D00D9121D00DEC1FD00BEA81
:100338001DD00D911BD00D9119D00FEF17D00AEADF
:1003480015D0935021F00D9111D09A95E1F7289A84
:1003580008954FEF11D000000000000000000000D9
:100368000000000000005A95A1F708950EBD0DB5D4
:1003780007FFFDCF0EB50895000000000000000043
:1003880000000000000000004A95B1F7089502E857
:100398002898ECDF00E0EADF289A007E003648F172
:1003A80000E22898E3DF00E0E1DF00E0DFDF08504B
:1003B8000993102F00E0DADF00E0D8DF00E0D6DF95
:1003C800099300E0D3DF00E0D1DF00E0CFDF09933D
:1003D80000E0CCDF0993135049F000E0C7DF00E0EC
:1003E800C5DF00E0C3DF09931A95D9F7289AD2FD33
:1003F800D2E020DF2EDF0F910FBF18950FB70F93B4
:100408000FE82898B3DF289A01E82898AFDF00E0C2
:10041800ADDF289A063139F0013129F00F31A1F307
:10042800023191F3B4CF07E82898A0DF00E09EDFFF
:10043800902E289A00E2289899DF00E097DF06506E
:100448000993102F0350002E00E090DF00E08EDFAC
:1004580000E08CDF09930130D9F000E087DF00E08D
:1004680085DF00E083DF00E081DF00E07FDF0993C4
:100478000A94D9F700E07ADF00E078DF00E076DF61
:10048800289A09939992D2FDD2E00F910FBF18953F
:1004980000E06CDF00E06ADF00E068DF00E066DFB4
:1004A80000E064DF09930A94D9F700E05FDF00E019
:1004B8005DDF00E05BDF289A09939992D0DEBADE0F
:1004C800D7DE2C9A00002C98249700E628984EDF57
:1004D8000BE04CDF01E64ADF08E848DF06E046DFCC
:1004E8000DEC44DF0BEA42DF099140DF09913EDF62
:1004F8000FEF3CDF0AEA3ADF289A2296D2FDD2E0D3
:100508000F910FBF1895A090C800A5FEFCCF2093AF
:10051800CE00089508E00093A10000E00093720067
:100528007FEFA0E018950FB70F938A9519F00F91F8
:100538000FBF189586B4002706BD7BD00FED00933A
:100548007A0084E00F910FBF18950FB70F93509062
:100558007800209079000F910FBF18955AD13BD1A0
:10056800709A00000000709800000000709A000067
:100578000000709800000000709A00000000709859
:1005880000000000709A0000000070980000000051
:10059800709A0000000070986C980000000000003D
:1005A800000000000000709A000000007098000031
:1005B8000000709A0000000070986C9A709A000011
:1005C800000070981CD16C9A709A00000000709816
:1005D80000000000709A0000000070980000000001
:1005E800709A00000000709800000000709A0000E7
:1005F8000000709800000000709A000000007098D9
:1006080000000000709A00000000709800000000D0
:10061800709A0000000070986C98000000000000BC
:10062800000000000000709A000000007098E7D0F9
:100638000895D1D0709A0000000070980000000062
:10064800709A00000000709800000000709A000086
:100658000000709800000000709A00000000709878
:1006680000000000709A0000000070980000000070
:10067800709A0000000070986C980000000000005C
:10068800000000000000709A000000007098000050
:100698000000709A000000007098B1D0EC9A08959C
:1006A8001FB71F9366F0EC9866D05ED0302E63D0EB
:1006B80056D0402E19D01F911FBF689418955BD053
:1006C80053D059D04CD0C02E07E0099303E00993CA
:1006D8005992299249923992C9928992D2FDD2E0CF
:1006E8001F911FBFE894189576D0709A00000000FB
:1006F800709800000000709A0000000070980000D8
:100708000000709A00000000709800000000709AC5
:1007180000000000709800000000709A00000000BF
:1007280070986C98000000000000000000000000B5
:10073800709A0000000070986C9A709A000000008F
:1007480070986C9800000000000000000000000095
:10075800709A00000000709852D0EC9A0895709A30
:1007680000000000709808956C9A709A00000000CC
:1007780070986C9808950027709A6499006870982A
:1007880000000000709A64990064709800000000EE
:10079800709A64990062709800000000709A6499D9
:1007A8000061709800000000709A64990860709861
:1007B80000000000709A64990460709800000000BE
:1007C800709A64990260709800000000709A6499A9
:1007D8000160709808956C98709800000000709AF5
:1007E8006C9A709800000000709A6C9800000000E5
:1007F800000000000000000070986C9A08956C9842
:100808006499FECF709A000000007098649BFECF38
:1008180008956C98709A000000007098000000001D
:10082800709A00000000709800000000709A0000A4
:100838000000709800000000709A00000000709896
:1008480000000000709A000000007098000000008E
:10085800709A00000000709800000000709A000074
:100868000000709800000000709A00000000709866
:1008780000000000709A000000007098000000005E
:10088800709A00000000709808950FB70F9300E069
:100898000093A5000093A4000091CE007F3F71F45F
:1008A8000F3F49F40FE209BB02E0009372000DE02C
:1008B8000093A10077270F910FBF1895772331F484
:1008C800AA270D93702F0F910FBF18950D937A9546
:1008D80091F7A0E00D91033038F0003428F40C9122
:1008E800083011F4A0E005DD08E00093A10000E065
:0C08F800009372007FEF0F910FBF189566
:00000001FF
